:020000040000FA
:040000008B01042844
:08000800850107309F008316FB
:1000100000308100003085000D308600831285019C
:1000200086010512A301A8017E24B922BE243C301A
:10003000A600B922A60B192805160130A924B92259
:1000400022217521231D2128FA22F02086192D282E
:10005000B92286192D282319F0207521FA220310C0
:10006000BA0C031C39287030BC070318BB0A1730C0
:10007000BB07A31C4628BA09BA0A3C08E03CBC00EE
:10008000031CBB0A3B082E3CBB00BA035A30BA071C
:100090003A08AE00AD010A3003213008413ECC00E1
:1000A0002E08303ECE00BB0CBC0CBB0CBC0C3F3051
:1000B000BB053C08AE003B08AD007D300321300895
:1000C000413ED000AD010310AE0D193003213008C0
:1000D000303ED200231C7728B509B50A3708703C9A
:1000E000B700031CB60A3608173CB600B5035A30F1
:1000F000B5073508AE00AD010A3003213008413E96
:10010000CD002E08303ECF000310B60CB70C3708D8
:10011000AE003608AD007D3003213008413ED100ED
:10012000AD010310AE0D193003213008303ED3006D
:100130008030A924231DD9282F212030A72417215E
:10014000C030A9244C30A7246F30A7246330A724E3
:100150002030A72464219430A9244C30A724613096
:10016000A7247430A7242030A7242030A7245321AB
:10017000D430A9244C30A7246F30A7246E30A72494
:100180002030A7243E21D330A9242030A724231DCA
:1001900026284708031D2628A80A0F302802031D19
:1001A0002628A801C6228D23D330A9245430A724A1
:1001B000262822212030A7242030A72422212030E5
:1001C000A7242030A724C030A9242030A724203021
:1001D000A72422212030A7242030A724222126284A
:1001E000C6228D234B236C23D330A9245530A7245A
:1001F000B922B922B922B922B922B922D330A9240D
:100200002030A7240800A000B001AF012008AE02F2
:1002100003180E29AD032D0903191229B00A031979
:10022000AF0A06292008AE070318AD0A08004508E2
:1002300074243A30A724460874243A30A724470887
:10024000742408004E30A7246F30A7242030A72440
:100250004730A7245030A7245330A724080048086B
:1002600074242030A724490800272030A7243230E6
:10027000A7243030A7244A08742408002030231A09
:100280003130A7243F087424DF30A72440087424A9
:100290002E30A724410874242730A7244530A31802
:1002A0005730A724080042087424DF30A7244308ED
:1002B00074242E30A724440874242730A7244E30F9
:1002C00023185330A72408004C08A7244D08A7245E
:1002D0004E08A7244F08A7245008A7245108A72494
:1002E0005208A7245308A7240800231D0516231924
:1002F0000512A03084009F22800024300002031DDC
:100300007B29840A9F2280000D300002031D812971
:10031000CB00A130840047300002031D7529840AF8
:1003200050300002031D7529840A52300002031D5B
:100330007529840A4D300002031D7529840A433053
:100340000002031D7529231D051223190516A90195
:10035000840A0D300002031908002C300002031D2E
:10036000A829A90A013029020319D3210230290240
:1003700003190522033029020319422204302902FD
:1003800003196D220530290203190F2206302902B4
:10039000031974220730290203197B22093029022C
:1003A0000319EC21A829840A000EF039C500840A3B
:1003B00000080F39C507840A000EF039C600840A08
:1003C00000080F39C607840A000EF039C700840AF6
:1003D00000080F39C7070800840A000EF039C8006A
:1003E000840A00080F39C807840A000EF039C900D2
:1003F000840A00080F39C907840A000EF039CA00C0
:10040000840A00080F39CA070800840A4130000234
:100410000319231556300002031923110800840A1A
:1004200000080F39AB002312031D2316840A000EA7
:10043000F039AC00840A00080F39AC072C08BF0063
:10044000AA01DD232E08BA00840A000EF039AB00A1
:10045000840A00080F39AB072B08C000840A840AFD
:10046000000EF039AC00840A00080F39AC072C08E4
:10047000C100AA01DD232E08BC00BE002D08BB0070
:10048000BD000800840A000EF039AC00840A0008A0
:100490000F39AC072C08C200AA01AB01DD232E08DE
:1004A000B500840A000EF039AB00840A00080F3949
:1004B000AB072B08C300840A840A000EF039AC0095
:1004C000840A00080F39AC072C08C400AA01DD23F8
:1004D0002E08B7002D08B6000800840A5330000229
:1004E0002310031923140800840A57300002A310B4
:1004F0000319A31408003030D600D700840A2E3028
:100500000002031D7E2A840A0008D40084038403A9
:100510000008D50084032C3000020319982A000833
:10052000D60084032C3000020319982A0008D70053
:10053000840A2C300002031D982A84030800061C3C
:100540009F2AB222061C9F2A0830A600A001B222D0
:10055000B22200000310061C0314A00CA60BA72A4D
:10056000200808004B30A40000000000A40BB42AAF
:100570000800FA30A500B222B222A50BBB2A08005F
:100580006430A500B222A50BC22A08002130C12385
:100590007730C1233030C1233030C123450E0F39AD
:1005A000303EC12345080F39303EC123B9222130E6
:1005B000C1237630C1233030C1233030C123460EF1
:1005C0000F39303EC12346080F39303EC123B922CE
:1005D0002130C1237530C1233030C1233030C123D5
:1005E000470E0F39303EC12347080F39303EC12333
:1005F000B92208000A30B000AF013508AE00AD01E5
:1006000009243608AD003708AE003C300321053020
:100610003007AE00AD010A3003213008B1070318DE
:10062000B20A231C182BB109B209B10A0319B20A84
:100630008430B1070318B20A0330B2073108B90099
:100640003208B8000A30B000AF013A08AE00AD0180
:1006500009243B08AD003C08AE003C3003210530C6
:100660003007AE00AD010A3003213008B10703188E
:10067000B20AA318402BB109B209B10A0319B20A90
:100680000830B1070318B20A0730B2073108BE00BC
:100690003208BD0008003908AE003808AD002F242C
:1006A000A430A9242B0874242C0874242130C123DD
:1006B0006C30C1232B0E0F39303EC1232B080F396C
:1006C000303EC1232C0E0F39303EC1232C080F3988
:1006D000303EC123B92208003E08AE003D08AD00FF
:1006E0002F24E430A9242B0874242C0874242130EE
:1006F000C1236B30C1232B0E0F39303EC1232B0891
:100700000F39303EC1232C0E0F39303EC1232C0847
:100710000F39303EC123B92208002130C1237A307D
:10072000C1233030C1233030C1234A0E0F39303E4F
:10073000C1234A080F39303EC123B9222130C123D9
:100740007930C1233030C1233030C123490E0F39F5
:10075000303EC12349080F39303EC123B922213030
:10076000C1237830C1233030C1233030C123480E3B
:100770000F39303EC12348080F39303EC123B9221A
:100780000800A0000830A6008614D223A00C03188D
:100790008610031C8614D223A60BC62B8610D223E8
:1007A000D2230800D32BD42BD52BD62BD72BD82B49
:1007B000D92BDA2BDB2BDC2B0800AD012A080F39F3
:1007C000AE00F8232B0E0F39AE07F8232B080F3994
:1007D000AE070318AD0AF8232C0E0F39AE07031825
:1007E000AD0AF8232C080F39AE070318AD0A08002C
:1007F0002D08A2002E080310AE0DAD0DAE0DAD0DEF
:10080000AE070318AD0A2208AD070310AE0DAD0DFB
:100810000800B101B201B301B4011030A600031009
:10082000AD0CAE0C031C1C2C3008B307031C1A2C97
:100830000130B4072F08B407B40CB30CB20CB10CE0
:10084000A60B0F2C0800A600A60803190800031029
:10085000B40CB30CB20CB10CA60B272C0800AA01E7
:10086000AB01AC011030A600AE0DAD0DAC0DAB0D63
:10087000AA0DA60B3C2C5B2C2A08033EA000A01955
:10088000AA002A08303EA000A01BAA002B08033EA5
:10089000A000A019AB002B08303EA000A01BAB00AD
:1008A0002C08033EA000A019AC002C08303EA0008C
:1008B000A01BAC00342C08002F242A080F39303E2E
:1008C000A7242B0E0F39303EA7242B080F39303EBA
:1008D000A7242C0E0F39303EA7242C080F39303EA8
:1008E000A7242030A7240800A100210E0F39303E94
:1008F000A72421080F39303EA72408000A30A6009B
:10090000C022A60B802C8612061203308500000040
:10091000861600008612C022861600008612C022AB
:10092000861600008612C02202308500000086165E
:100930000000861200002830A9241C30A9240C30A5
:10094000A9240430A9240130A924B92208000616DC
:10095000AA2C0612A000200E0F3985000000861672
:1009600000008612000020080F398500000086165E
:100970000000861200000000B22208008030A92486
:100980004730A7245030A7245330A7242030A72471
:100990004E30A7244D30A7244530A7244130A7244A
:1009A0002030A7242F30A7242030A7244430A724A8
:1009B0005230A7244930A7244130A7244330A7242C
:1009C0005330A7242D30A7244730A7243230A72442
:1009D000C030A9244930A7246E30A7247430A7243E
:1009E0006530A7247230A7246630A7246130A7247D
:1009F0006330A7246530A7249430A9244730A72466
:100A00003430A7244A30A7244E30A7245430A724DA
:100A1000D430A9244130A7247530A7246730A724F7
:100A20002030A7243230A7243030A7243130A72427
:100A30003030A72408005430C1236530C1237330FF
:100A4000C1237430C1232030C1236D30C1236530F0
:100A5000C1237330C1237330C1236130C123673098
:100A6000C1236530C1232030C1234030C123203051
:100A7000C1233130C1233130C1233530C12332305D
:100A8000C1233030C1233030C1232030C123423054
:100A9000C1236130C1237530C1236430C1232030AC
:0A0AA000C1230D30C1230A30C12329
:100E0000A10007308A000030211A0A3021070F396B
:100E1000A100A1030310210DA107A60121082607A7
:100E20001827A724A60A03302602031908000E2F4C
:100E300082074A3461346E344634653462344D344A
:100E4000613472344134703472344D3461347934E5
:100E50004A3475346E344A3475346C3441347534E4
:100E600067345334653470344F34633474344E34DF
:0A0E70006F34763444346534633483
:084000000D0000000B0001009F
:02400E00623F0F
:00000001FF
